:1000000020000120D3020000D1020000D102000034
:10001000D1020000D1020000D10200000000000067
:10002000000000000000000000000000D1020000FD
:10003000D102000000000000D1020000D102000047
:10004000D1020000D1020000D1020000D102000064
:10005000D1020000D1020000D1020000D102000054
:10006000D1020000D1020000D1020000D102000044
:10007000D1020000D1020000D1020000D102000034
:10008000D1020000D1020000D1020000D102000024
:10009000D1020000D1020000D1020000D102000014
:1000A000D1020000D1020000D1020000D102000004
:1000B000D1020000D1020000D1020000D1020000F4
:1000C000D1020000D1020000D1020000D1020000E4
:1000D000D1020000D1020000D1020000D1020000D4
:1000E000D1020000D102000000000000000000006A
:1000F00000000000D1020000D1020000D102000087
:10010000D1020000D1020000D1020000D1020000A3
:10011000D1020000D1020000D1020000D102000093
:10012000D1020000D1020000D1020000D102000083
:10013000D1020000D1020000D1020000D102000073
:10014000D1020000D1020000D1020000D102000063
:10015000D1020000D1020000D1020000D102000053
:10016000D1020000D1020000D1020000D102000043
:10017000D1020000D1020000D1020000D102000033
:10018000D1020000D1020000D1020000D102000023
:10019000D1020000D1020000D1020000D102000013
:1001A000D1020000D1020000D1020000D102000003
:1001B000D1020000D1020000D1020000D1020000F3
:1001C000D1020000D1020000D1020000D1020000E3
:1001D000D1020000D1020000D1020000D1020000D3
:1001E000D1020000D1020000D1020000D1020000C3
:1001F000D1020000D1020000D1020000D1020000B3
:10020000D1020000D1020000D1020000D1020000A2
:10021000D1020000D1020000D1020000D102000092
:10022000D1020000D1020000D1020000D102000082
:10023000D1020000D1020000D1020000D102000072
:10024000D1020000D1020000D1020000D102000062
:10025000D1020000D1020000D1020000D102000052
:10026000D102000010B5054C237833B9044B13B10B
:100270000448AFF300800123237010BD000000206C
:1002800000000000380400000C4B43B10C480D493D
:1002900010B5AFF300800C48036823B910BD0A48BD
:1002A000036833B97047094B002BF7D0BDE8104005
:1002B0001847064B002BF5D0184700BF0000000080
:1002C0003804000004000020380400000000000092
:1002D000FEE708B50F4A104B9A420ED10F4B104A59
:1002E0000021934212D30F4B0F4A23F07F039360F8
:1002F00000F06EF800F01CF8FEE70C49043A8B425F
:10030000ECD252F8040F43F8040BF8E743F8041B4F
:10031000E7E700BF380400000000002000000020D4
:100320001C0000200000000000ED00E000000020A4
:10033000244B5A6942F400425A615A69042161F31C
:10034000CE225A615A6942F4C0625A615A696FF307
:10035000C7125A615A690A435A615A6942F0020245
:100360005A611A69D207FCD55A6B6FF314425A636B
:100370005A6B772161F30C025A639A6B052161F382
:100380001A429A639A6B022161F347129A6393F8B7
:1003900030206FF3C71283F8302093F830200A43DF
:1003A00083F83020074B1A6CD007FCD51A6C9107E4
:1003B000F9D5054B054A1A625A685207FCD400BFAA
:1003C000FEE700BF00100040001C004007010100D4
:1003D00070B50D4E0D4CA41BA4100025A54209D1EB
:1003E0000B4E0C4C00F018F8A41BA4100025A542DD
:1003F00005D170BD56F8253098470135EEE756F81F
:10040000253098470135F2E7240400002404000059
:100410002404000028040000F8B500BFF8BC08BCA4
:100420009E46704789020000F8B500BFF8BC08BCC2
:080430009E46704765020000C2
:00000001FF
